:100000000C94B4040C94DC040C94DC040C94DC0418
:100010000C94DC040C94DC040C94DC040C94DC04E0
:100020000C94DC040C94DC040C94DC040C94872BFE
:100030000C94DC040C94DC040C94DC040C94DC04C0
:100040000C94ED2B0C94DC040C94DC040C94DC0478
:100050000C94DC040C94DC040C94DC040C94DC04A0
:100060000C94DC040C94DC04A817AB17AE17B11782
:10007000B417B717BA17BD17C017121B1C1B491BA3
:10008000561B981BA51B001C161BC21B4C1BF01BF0
:10009000040460F06090040490F060900404F0F0B8
:1000A0006090040460606090180A30900078F0005E
:1000B0003060C04890200000400000007860407828
:1000C0006000306000489000150C00000000000047
:1000D000000000C00018F00038F80078C1FC78FB80
:1000E00006F8FC01F8F800F8F800F8F800F8150C2C
:1000F00000000030000044D30052AA0076A900009E
:1001000000001800001D56301555501D9560000068
:1001100000AAAAA8150C007FF80013F80001F80047
:1001200001380400386C0018FE0038FF80B8FF0169
:10013000F8FE01F8FF00F8FFFFF8150C00000000C2
:10014000000000010001030001960000BC1000F84F
:1001500010807010807838C07878E47878FFFFF8E5
:10016000150C00000000000000450081FF80C7FF63
:10017000C0E3FFE0C1FFC0F09380F80000FC000086
:10018000FE0000FFFFF8150C00000000000099F0D1
:100190000065D800F07E0048CF00400F804017C0B7
:1001A000500360E00638FFFFF8FFFFF8150C000071
:1001B00000060A000F84000700F000001020007005
:1001C0007000F0F80190200290FC0490F8FFF8F322
:1001D000FFF8150C0000000001C00003E00002A0C1
:1001E0000203E00601C04580804783E03D0C803C6F
:1001F000F1C0240140FFFFF8150C000000000000D2
:10020000000000800008C0009880DBF881FFF880C3
:100210007FF8802FF8C007F8F80FF8FFFFF8150CEB
:1002200007C03807E01807801803000803800003A0
:100230000400810400C00C00E00E00F01E00E0FF8E
:1002400080FFFFF8150C0000000000000000000017
:100250000000000008400018E00078E00038C0000E
:1002600038E00078F109F8FFFFF8150C00000000F5
:10027000000001C060E00000000E00070000006008
:10028000C03000300007001E0000001C18E0000015
:10029000150C000000FF9FF8FFCFF880E608EFF391
:1002A000D8C07008FDE4F880CE78DF9F38C03FB832
:1002B000FFFF88FFFFB8150C0000000000000000E1
:1002C00000F00000F80000F80000FC0018FC0078C6
:1002D000FC0FF8FE1FF8FFFFF8FFFFF8150C0000F9
:1002E000000000701F00302880702840307FF070C0
:1002F000FFF830CF38104F301030C010FFFFF8FF3C
:10030000FFF8150C0000000000000FFFF880080047
:10031000F0FF00CFE4804FE64030FFE0007FC000F8
:100320001110007FE0000000150C0000000000002C
:1003300001C00000E00007FC0001FE0002ABF01F5E
:10034000FFE01FFFC01FFF80AFFFA8555550150CE1
:10035000000000000000801000C01800C00808C0A5
:100360001C38C21C78C61C78E61C78F61C78FF3F47
:10037000F8FFFFF8150C01E03800F018487808FC89
:100380003F88FC3FC0F87F80F07F00F0F600D0404F
:1003900008900018800078FFFFF8150C000000009E
:1003A00000000000400001C09001E8FC03E8FE07E7
:1003B000F8F00FF8E007F8C003F8F807F8FFFFF8C7
:1003C000150C00000000200000200000200000703C
:1003D00000005000445110EEFBB8EEDBB8458D1024
:1003E000FFFFF8FFFFF8150C00028000AB800071E2
:1003F00000007100007300002600007C0000F8007F
:1004000000F00000700000F000FFFFF8150C000085
:100410000000000000A8000050001FFFC01FFFC028
:100420000A8A80FA8AF8AA8AA8AA8AA8AA8AA8FFA9
:10043000FFF8150C0000000000001808203C0440E4
:100440007E0FE0DB1BB0FF3FF8242FE85A2828A5D9
:1004500006C0000000FFFFF8150C0000001F0000A0
:100460003F83C07B07E07E0FF07C0C907E0DB07F59
:100470000FF03F8FF01F0A50000000FFFFF8150C2F
:100480000000380000104011383004007AAA003013
:100490000400401170000020000870801C00C03E65
:1004A00008FFFF780404F0F0F0F00404E0F0F0F04E
:1004B000040460F0F0F0040470F0F0E0040460F074
:1004C000F070040460F0F060040400000000040414
:1004D00010000000040490000000040480000010DC
:1004E0000404900000800404900000904823000061
:1004F000008254000000000000015B15B500000000
:10050000000001D255250000000000015154A30055
:10051000000000000000000100000000000FFFFFCD
:10052000FA6000000000000000000000000014005D
:1005300000000128000000155A4C14C2A3600000FE
:100540001D552A1483AA50000015956A0982A950E6
:10055000000000000000000000000000000000009B
:1005600000FF8000000000000003FFE0000E00001C
:10057000000007FFE00031800000000FFFF00040A6
:10058000400000000FFFF0008F200000000FFFF080
:100590000090A00000000FFFE0013FD00000000F1E
:1005A000FFC0013FD0000000027F800165500000C5
:1005B000000FFE0003E0500000000FFC00056690F5
:1005C0000000000FFE0006B0A00000000A8F8005AA
:1005D0005F600000000007C003AAA0000000003F09
:1005E000F00475600001F001FFF8050FC010011B59
:1005F000C1FFF808C3FFF8000FFCFEF80837FCF84D
:10060000007FFCFDE80A0FFFF00007BF67D81180EC
:100610003FF0021E53FF781078148003F3EFFDF0D3
:100620002007F3000000FFF7F00A4E6F205344202C
:1006300063617264206F720A6E6F204C4F414445B3
:10064000522E4845580A0A153A45786974001D200B
:10065000466C617368696E670A20206C6F6164651F
:10066000722E2E2E0A0A444F4E2754205455524EB5
:10067000204F464621000A0A153A49676E6F726597
:10068000006D560A0A504C45415345205455524E70
:10069000204F464620004C4F57204241545445526B
:1006A00059212000172B152010204C4F4144455252
:1006B00000172B162013140017534400161378004C
:1006C00016131400151020001520100000540A0302
:1006D000E181867F3E186D830F0F0E0183866033A4
:1006E000186DC3198F1803C38E6033186DE330CFB4
:1006F0001803C39E603630CDE360CF3006C79E7EC0
:100700003E30CDB360CF300CC6F6603330D9B66022
:10071000CF33CFCCF66061B0DB1E60CF30D86CE653
:10072000C061B0DB1E618F19986CC6C063B19B0EAF
:10073000330F0FB078C6FF7E1F1B061E0F05008902
:10074000300802380249786814000003053F213F51
:100750001208120A100A0E1C0E0C1E0C141A141683
:100760001F161E131E1E1B1E1E1F1E3F213F3A2F4B
:100770003A173D173F213F181F02040A041F0E04B9
:10078000040E1F0A1F0A0E0E1F04110E2E252E2FF7
:100790002A2E262929021F02081F08150E04040EFE
:1007A000150E15151B151B040604040C040000008F
:1007B0000017000300031F0A1F16371A1904130A33
:1007C000153A000300000E11110E000A040A040E6F
:1007D000040030000404040010001804031F111F5B
:1007E000121F101D151711151F07041F17151D1FA8
:1007F000151D01011F1F151F17151F000A000032CC
:1008000000040A110A0A0A110A040115020E11173E
:100810001E051E1F150A0E110A1F110E1F15111F8E
:1008200005010E111D1F041F111F1108100F1F04B9
:100830001B1F10101F061F1E040F0E110E1F09068E
:100840000E112E1F051A121509011F011F101F0F6F
:10085000180F1F0C1F1B041B031C03191513001F6B
:1008600011030418111F00020102202020000102C0
:100870000C121E1F120C0C12120C121F0C1A140454
:100880001E05242A1E1F021C141D1020201D1F08D7
:1008900014111F101E041E1E021C0C120C3E0A0412
:1008A0000C123E1E040214160A020F120E101E0E27
:1008B000100E1E081E120C1226281E322A26041E96
:1008C00021001F00211E040102013F213FF6E8DB49
:1008D000CFC3B8AEA49B928A827B746E68625C5769
:1008E000524E4945413E3A3734312E2C2927252393
:1008F000214500680100000500380168010000077B
:100900000903090101FF030101F7030000000800CA
:1009100002010000030407000000000000000001C5
:100920000204081020408001020408102001020483
:100930000810200404040404040404020202020255
:100940000203030303030300000000230026002921
:100950000000000000250028002B000000000024FB
:100960000027002A0000091C11241FBECFEFD8E089
:10097000DEBFCDBF12E0A0E0B1E0ECE3F5E602C0DF
:1009800005900D92A23BB107D9F727E0A2EBB2E0A8
:1009900001C01D92A730B207E1F719E0C8E6D9E01F
:1009A00004C02297FE010E941932C636D107C9F74A
:1009B0000E94ED2F0C949C320C9400008435D8F4E6
:1009C0006033C8F4962F959595959595E82FFF2758
:1009D000E7FDF095E850FB4F84E59802E00DF11D2E
:1009E0001124808190E0677002C0959587956A9583
:1009F000E2F78170089580E008950F931F93CF93DD
:100A0000DF93FC01862F643508F044C0403308F0C2
:100A100041C090A1042F059505950595C62FDD27AA
:100A2000C7FDD095142F1770923031F4642F0E94B7
:100A3000DE048823F1F00AC0933031F44627848520
:100A4000482740FF03C015C0911113C0FE0184E583
:100A50000802E00DF11D1124E850FB4F81E090E009
:100A6000012E01C0880F0A94EAF78095908198239F
:100A700010C0FE0184E50802E00DF11D1124E850CC
:100A8000FB4F81E090E001C0880F1A95EAF7908152
:100A9000982B9083DF91CF911F910F910895CF9361
:100AA0006CEE74E080E794E00E94FB1F10928804D3
:100AB000C1E0C093C7031092C4038AE18093C603C8
:100AC00084E18093BE021092C6021092B30225E127
:100AD00030E040E050E060E070E0CB010E94892F00
:100AE0006093BD0282E08093B80283E08093B902F4
:100AF000C093B7028093B602C093B202CF9108951B
:100B000080E794E00E9477200C944F056F927F92CB
:100B10008F929F92AF92BF92CF92DF92EF92FF920D
:100B20000F931F93CF93DF93CDB7DEB765970FB6C3
:100B3000F894DEBF0FBECDBF40E025E130E0842F4A
:100B400090E0E1E0F0E0EC0FFD1FE80FF91F880FE7
:100B5000991F880F991FB9010E94C23180834F5F8E
:100B6000453168F34093C50225E130E040E050E0B4
:100B700060E070E0CB010E94892F1092C50220E056
:100B800070E085E190E0861B970BE22FF0E02F5F8D
:100B9000E817F9079CF4A1E0B0E0AC0FBD1FAE0F61
:100BA000BF1F3C91E60FF71F41E050E04C0F5D1F67
:100BB000E40FF51F40814C933083E7CF1092C502BC
:100BC00089E0C82EBB24B3949AE0A92E2BE0D22E44
:100BD0008091C502282F30E06091B902E091B802FF
:100BE0004E2F50E06E9FF00111242E173F070CF09E
:100BF000DCC0C29EF001C39EF00D1124E052FC4FF8
:100C000013829091B60297830E9494318483158257
:100C1000168290E06091B702461B51098417950730
:100C20000CF0B682C29E8001C39E100D11240052AA
:100C30001C4FD80118961C921897E1E0F0E0EC0FD9
:100C4000FD1FE20FF31F8080882D880F880FF801A9
:100C5000819399249394980C80FC1FC011961C9248
:100C60007F01F7017080FAE0F7150CF444C06624A8
:100C70006394670C662D892D0E94DE04811138C0B3
:100C800062E0670D892D0E94DE04813089F5770CC2
:100C9000770CD80111967C921AC0D8011196AC92AB
:100CA0007F01F70170801714ACF561E0670D892DA5
:100CB0000E94DE0481112AC062E0670D892D0E9426
:100CC000DE04813019F5770C770CF8017182809180
:100CD000C502C89EF0011124E052FC4F9081993268
:100CE00014F0128201C0B2828F5F8093C50270CF70
:100CF000F7016082B6CF882D6D2D0E949431892F27
:100D0000880F880FD80111968C930DC07A94D70163
:100D10007C92C7CF882D6D2D0E949431892F880F2A
:100D2000880FF801818361E0690F892D0E94DE043C
:100D300081111BC061E08EEB94E00E948C228091B7
:100D4000C502E1E0F0E0EC0FFD1FE80FF11D20818E
:100D5000822F6D2D0E9494319E5F61E0620F492FBA
:100D60008EEB94E00E94FD04B2CF60E08EEB94E045
:100D70000E948C228091C502E1E0F0E0EC0FFD1FA3
:100D8000E80FF11D2081822F6D2D0E9494319F5F0D
:100D900061E0620F492F8EEB94E00E94FD0461E058
:100DA0008EEB94E00E948C2292CF65960FB6F89459
:100DB000DEBF0FBECDBFDF91CF911F910F91FF908E
:100DC000EF90DF90CF90BF90AF909F908F907F90EB
:100DD0006F9008958091BA028530D1F0863069F025
:100DE000843011F5E091BB0299E0E99FF0011124F4
:100DF000E052FC4F9181915015C0E091BB0299E007
:100E0000E99FF0011124E052FC4F918193500AC0F8
:100E1000E091BB0299E0E99FF0011124E052FC4F00
:100E200091819250918302C0882319F08150809360
:100E3000BA0208952F923F924F925F926F927F92E3
:100E40008F929F92AF92BF92CF92DF92EF92FF92DA
:100E50000F931F93CF93DF93CDB7DEB728970FB6CD
:100E6000F894DEBF0FBECDBF1092C4024090B9020D
:100E70008091B802489E20011124E9E03E2E909115
:100E8000C4029983092F10E0041515050CF0C4C0A5
:100E9000309EC001319E900D112480529C4F988746
:100EA0008F836C019FEFC91AD90AAF81B88511965B
:100EB0009C9111979C5FFC90692F8F2D9E830E94BF
:100EC000DE049E81811190C0692F83E08F0D0E9406
:100ED000DE04811189C01092C3028F80988474014E
:100EE000A5E0EA0EF11C5401B3E0AB0EB11C3401D5
:100EF000E4E06E0E711CC40107969B838A83F701A0
:100F000060812090C302462F50E0822D90E0481768
:100F10005907C4F1F601908154E0590FD4014C9166
:100F2000652F842F4D835C839E830E94DE044D8158
:100F30005C81811123C0652F83E0840F0E94DE0451
:100F40009E8181111BC091330CF457C0F501808143
:100F5000811114C0D301EC91F0E0EE0FFF1FE852B5
:100F6000FC4F8081815080831092B502EA81FB8121
:100F70001082D7011C9281E0F50180832394209296
:100F8000C302BDCF643050F4AF81B88513968C9105
:100F90001397811103C06F5F15966C93309E5001BB
:100FA000319EB00C1124F501E052FC4F5F01F1803D
:100FB00063E0D62EDF0CE0806D2D82E08E0D0E9466
:100FC000DE048130F1F06D2D81E08E0D0E94DE0493
:100FD000813029F4D50113968C91882391F0898171
:100FE0008F5F8093C4024BCF309EF001319EF00D95
:100FF0001124E052FC4F1582D1CF9F5FD6019C9304
:10100000BDCF309EF001319EF00D1124E052FC4F17
:10101000FA94F1821582E3CF28960FB6F894DEBFDA
:101020000FBECDBFDF91CF911F910F91FF90EF9039
:10103000DF90CF90BF90AF909F908F907F906F90F8
:101040005F904F903F902F9008951F93CF93DF9321
:101050006091B9028091B802689FB001112420917B
:10106000D40330E04091D50350E0C091BE02B0916E
:10107000B502A0E0D9E011E08A2F90E0861797072B
:10108000A4F5D89FF001D99FF00D1124E052FC4F38
:101090008381811128C08081992787FD9095281729
:1010A00039070CF1049682179307ECF08181992798
:1010B00087FD909548175907B4F004968417950753
:1010C00094F087818150878381110CC01383E48160
:1010D000F0E0EE0FFF1FE852FC4F808181508083CB
:1010E000B0E001C0C087AF5FC7CFB093B502A09397
:1010F000C502DF91CF911F9108952091B80280E041
:1011000090E0821758F4E82FF0E0EE0FFF1FE8524E
:10111000FC4F308131119F5F8F5FF3CF8093C50209
:10112000923018F487E08093C70308951F93CF93FC
:10113000DF93C091B802D0E08091BC0290E00196AC
:10114000BE010E94C2319C01220F331FF901E852F7
:10115000FC4F5081552391F38093BC02C091B9029A
:101160008C9F402D1124D0E0818119E090E0019600
:10117000BE010E94C231942F980F199FF0011124D3
:10118000E052FC4F53815111F1CFD901A852BC4F0D
:1011900011968C939093BB028091BE02808710922F
:1011A000B50284E08093B40282E08093D1038AE0A8
:1011B0008093D2031092D3038093C703DF91CF9122
:1011C0001F910C947D083091D60323E0832F622F6A
:1011D0000E94A0319091D403890F8093D403409151
:1011E000D703842F622F0E94A0319091D503890FDD
:1011F0008093D5032091B202240F2093D703632F4D
:10120000772767FD709577FF03C071956195710928
:101210006D30710544F04CE03402C00111240E948D
:10122000C2316093D603622F772767FD709577FFF1
:1012300003C07195619571096D30710544F03CE012
:101240002302C00111240E94C2316093D703089584
:10125000CF932091D403253530F44091D5038FEC02
:10126000840F833318F4CF910C949608E22FE695FF
:10127000E6958CE0E89FF0011124842F86958695F1
:10128000E80FF11DE953FD4F80818C3318F486E09F
:101290008093C7036091B9028091B802689FB00142
:1012A0001124B091C703A0E0C9E030E050E08A2FDC
:1012B00090E08617970704F5C89FF001C99FF00DCD
:1012C0001124E052FC4F8081992787FD90952817C3
:1012D000390784F004968217930764F08181992777
:1012E00087FD9095481759072CF0049684179507A9
:1012F0000CF0B6E0AF5FDBCFB093C703A093C5029D
:10130000CF9108955091C80390E070E04091CA03D6
:101310002091CD033091CC035C3308F097C05CE0A2
:10132000589FF001599FF00D1124E60FF71FE95364
:10133000FD4F10824C3340F05091CB035C3320F0D2
:101340002C3310F05AE050833C33A0F05091CE0380
:101350005C3380F05091CF035C3360F05CE0589FC9
:10136000F001599FF00D1124E60FF71FE953FD4FCF
:101370005BE050832C3398F05091CF035C3378F0CE
:101380005091D0035C3358F05CE0589FF001599FB6
:10139000F00D1124E60FF71FE953FD4F50835091D4
:1013A000C9035C33A8F04C3398F03C3360F0ACE0F8
:1013B000A89FF001A99FF00D1124E60FF71FE95334
:1013C000FD4FADE0A083E091CB03EC3308F059C1B1
:1013D0003C33D0F02C33C0F0E091CE03EC33A0F0DE
:1013E000E091CF03EC3380F0E091D003EC3360F078
:1013F000ACE0A89FF001A99FF00D1124E60FF71FA4
:10140000E953FD4FA5E1A0834C3308F432C1A0910C
:10141000CB03AC3308F4A8C02C3308F4A5C0E0918A
:10142000CF03EC3308F4A0C0E091D003EC3308F410
:101430009BC0BCE0B89FF001B99FF00D1124E60FEE
:10144000F71FE953FD4FB6E1B0838EC05CE0589FB3
:10145000F001599FF00D1124E60FF71FE953FD4FDE
:101460005CE350834C3320F42C3310F456E4508367
:101470003C3380F45091CF035C3360F45CE0589FC0
:10148000F001599FF00D1124E60FF71FE953FD4FAE
:1014900057E450832C3380F45091CF035C3360F4D5
:1014A0005CE0589FF001599FF00D1124E60FF71FE3
:1014B000E953FD4F58E450834C3380F43C3340F5FE
:1014C0005CE0589FF001599FF00D1124E60FF71FC3
:1014D000E953FD4F2C3330F450E505C03C3308F49C
:1014E0001CC1089559E450832C3320F55091CF034B
:1014F0005C3308F0C2C05CE0589FF001599FF00DCA
:101500001124E60FF71FE953FD4F51E55083B5C095
:101510002C3380F44091CF034C3360F44CE0489F6F
:10152000F001499FF00D1124E60FF71FE953FD4F1D
:1015300042E540833C33B8F43091CF033C3308F0AC
:10154000EFC03CE0389FF001399FF00D1124E60F09
:10155000F71FE953FD4F83E580832C3308F0E0C08B
:101560008EE68083089508955C33F0F04C3308F4E0
:10157000D7C03C33A0F0E091CE03EC3380F0E09193
:10158000CF03EC3360F0BCE0B89FF001B99FF00DE1
:101590001124E60FF71FE953FD4FB7E1B083AC33D9
:1015A00018F03C3308F080C0AC33E0F03C33D0F0AE
:1015B0002C33C0F0E091CE03EC33A0F0E091CF03E8
:1015C000EC3380F0E091D003EC3360F0ACE0A89F06
:1015D000F001A99FF00D1124E60FF71FE953FD4F0D
:1015E000A9E2A0835C3308F49BC04C3308F498C094
:1015F0004091CB034C33D8F03C3308F46FC02C330C
:1016000008F46CC05091CF035C33B8F05091D00314
:101610005C3398F05CE0589FF001599FF00D112465
:10162000E60FF71FE953FD4F5AE2508306C03C33E3
:1016300008F454C02C3308F451C05091CE035C33ED
:1016400008F44CC05091CF035C3308F447C050916C
:10165000D0035C3308F442C05CE0589FF001599F0E
:10166000F00D1124E60FF71FE953FD4F5BE25083A5
:1016700035C05C3308F054C0B5CF4C3308F050C0CF
:1016800049CF3C3308F4C3CE2C3308F4A3CEACE0EE
:10169000A89FF001A99FF00D1124E60FF71FE95351
:1016A000FD4FA4E1A08396CE2C3308F47DCFE091CA
:1016B000CE03EC3308F478CFE091CF03EC3308F499
:1016C00073CFBCE0B89FF001B99FF00D1124E60F75
:1016D000F71FE953FD4FB8E2B08366CF4C33E0F01B
:1016E0003C33F0F02C33E0F02091CE032C33C0F0EB
:1016F0002091CF032C33A0F02091D0032C3380F025
:101700002CE0289FF001299FF00D1124E60FF71F10
:10171000E953FD4F82E325CF08952C3308F4E6CE3C
:101720000895DF92EF92FF920F931F93CF93DF9371
:1017300081E08093C502DD24D394CCE38091C5027F
:101740008D3008F086C0D092C4021091C402D091AE
:10175000C502163108F079C06D2F812F0E94DE047A
:10176000882319F01092C80302C0C093C803EE2466
:10177000EA94ED0E0FEF010F6E2D802F0E94DE0414
:10178000882319F01092C90302C0C093C9036E2DBB
:10179000812F0E94DE04882319F01092CA0302C030
:1017A000C093CA03FF24F394F10E6E2D8F2D0E9477
:1017B000DE04882319F01092CB0302C0C093CB0340
:1017C0006D2F802F0E94DE04882319F01092CC0325
:1017D00002C0C093CC036D2F8F2D0E94DE0488239E
:1017E00019F01092CD0302C0C093CD03EE24E39410
:1017F000ED0E6E2D802F0E94DE04882319F01092CA
:10180000CE0302C0C093CE036E2D812F0E94DE0452
:10181000882319F01092CF0302C0C093CF036E2D1E
:101820008F2D0E94DE04882319F01092D00302C08D
:10183000C093D0036FEF6D0F802F0E9482098091BB
:10184000C4028F5F8093C40280CFDF5FD093C50254
:1018500075CFDF91CF911F910F91FF90EF90DF90A7
:1018600008950F9360E08EEB94E00E948C220CE0D0
:1018700025E140E060E08EEB94E00E94022361E00D
:101880008EEB94E00E948C220EE027E140E060E0C5
:101890008EEB94E00E94DA222091C30386E2289F17
:1018A0009001112428533F4F41E061E08EEB94E01A
:1018B0000E9422250E9486050E94910B60E08EEB1B
:1018C00094E00E948C2227E140E060E08EEB94E0FF
:1018D0000E94022361E08EEB94E00F910C948C2225
:1018E0000F931F93CF93DF935091D6034091D7036B
:1018F0007091D4036091D50357FD74C047FD39C082
:10190000172F16951695212F30E0F9013197C62F24
:10191000C695C6958C2F90E00CE00E9FD0010F9FCE
:10192000B00D1124A80FB91FA953BD4FEC91EC3392
:1019300008F0E5C0029FF001039FF00D1124E80FAD
:10194000F91FEA53FD4F00810C3308F0D8C0852FF2
:10195000992787FD9095552747FD509555954795B3
:10196000481759070CF075C01150163108F0D7C050
:10197000BCC0C72FC695C6952C2F30E0F901319712
:10198000862F8695869590E01CE01E9FD0011F9FB4
:10199000B00D1124A80FB91FA953BD4FEC91EC3322
:1019A00008F0ADC0129FF001139FF00D1124E80F55
:1019B000F91FE853FD4F10811C3308F0A0C0252FFC
:1019C000332727FD3095552741950CF450955595B3
:1019D0004795421753070CF08DC0C150C63108F02F
:1019E0009EC083C047FD4CC0872F8695869590E0AA
:1019F000FC013196C62FC695C6952C2F30E01CE011
:101A00001E9FD0011F9FB00D1124A20FB31FA95319
:101A1000BD4FEC91EC3328F5189FF001199FF00DA4
:101A20001124E20FF31FEA53FD4F10811C33C8F459
:101A3000052F112701950CF41095552747FD50955A
:101A4000559547954017510724F445970CF067C00A
:101A50004CC0783508F063C0C150CD3008F45DC08B
:101A60005EC0783508F05BC0643308F058C04CE0C5
:101A7000489FF001499FF00D1124E20FF31F4BC066
:101A8000272F2695269530E0F9013196862F8695E9
:101A9000869590E0CCE0CE9FD001CF9FB00D112471
:101AA000A80FB91FA953BD4FEC91EC3340F5C29F6D
:101AB000F001C39FF00D1124E80FF91FE853FD4F0B
:101AC000C081CC33E0F4C52FDD27C1950CF4D0954F
:101AD0008E01552741950CF4509555954795401723
:101AE000510744F425313105D4F46433C0F48CE358
:101AF0008C9315C0783598F40C978CF40EC078351B
:101B000070F4643360F44CE0429FF001439FF00DA9
:101B10001124E80FF91FE953FD4F8CE380831092E5
:101B2000C502CCE08091C5028C3008F0C6C010928E
:101B3000C4028091C4026091C502853108F0B9C029
:101B4000462F50E0282F30E0FA01C89FE00DF11D2C
:101B50001124E953FD4F90819093C803882389F0A5
:101B6000662379F0D9011197CA9FF001CB9FF00D40
:101B70001124E40FF51FEA53FD4F90819093C903A0
:101B800004C01092C903662389F0DA011197C29F3D
:101B9000F001C39FF00D1124EA0FFB1FE953FD4F25
:101BA00090819093CA03843121F415C01092CA0326
:101BB00012C0662381F089010F5F1F4FC09FF001A3
:101BC000C19FF00D1124EA0FFB1FE953FD4F9081D7
:101BD0009093CB0302C01092CB03882389F0D901E4
:101BE0001197CA9FF001CB9FF00D1124E40FF51F50
:101BF000E953FD4F90819093CC038431A1F002C052
:101C00001092CC03D9011196CA9FF001CB9FF00D21
:101C10001124E40FF51FE953FD4F90819093CD03FC
:101C20008823A1F002C01092CD036B3078F4D90163
:101C30001197CA9FF001CB9FF00D1124E953FD4F7E
:101C4000E40FF51F91819093CE0304C01092CE0350
:101C50006B3088F44F5F5F4FC29FF001C39FF00D60
:101C60001124E40FF51FE953FD4F90819093CF03AA
:101C7000843121F414C01092CF0311C06B3078F47A
:101C80002F5F3F4FC29FF001C39FF00D1124E40F5F
:101C9000F51FE953FD4F90819093D00302C010923D
:101CA000D0030E9482098091C4028F5F8093C40296
:101CB00040CF6F5F6093C50235CFDF91CF911F9109
:101CC0000F910895DF92EF92FF920F931F93CF939E
:101CD000DF938091B302882311F0815059C1809124
:101CE000D303811139C11092C502C9E00CE0809183
:101CF000C502823008F028C188E08093C4021AE04F
:101D0000D1E08091C402882309F418C11092C30263
:101D100024E1F22EE090C3024091C40289E08E15C6
:101D200008F408C11092BF02E091BB028091C50285
:101D3000282F30E0220F331F2150310931E0380FB6
:101D4000CE9FF0011124E052FC4F8081380F50E00B
:101D5000DA01AE57BD4F8C91612F0E94A031A82FA0
:101D6000829F300D11243093D40391819F5F980F8F
:101D70009093D503E694FA01E557FD4F8081612FDA
:101D80000E94A031829F202D11242E9D202D1124F0
:101D90002093D603AE9DE02C1124E092D7038091CE
:101DA000BF028111C1C01092C2024091C20250E034
:101DB0009091B9028091B802989FC00111244817F0
:101DC00059076CF7C49FF001C59FF00D1124E05234
:101DD000FC4F8081992787FD9095E090D4032E2DAC
:101DE00030E0BC0164507109D090D5032617370745
:101DF0000CF478C00896821793070CF473C06181C5
:101E0000772767FD70958D2D90E0DB0114978A1779
:101E10009B070CF467C0685F7F4F681779070CF465
:101E200061C0638161115EC06091BB0270E0C69FBA
:101E3000D001C79FB00D1124A052BC4FF48114965D
:101E4000EC911497FE1709F44DC0E091D303E11112
:101E500047C0E1E0F091C502F11101C0E0E0129647
:101E6000EC93E091C402E093D103E091C302E093CC
:101E7000D203C49FF001C59FF00D1124E052FC4F26
:101E80004081552747FD5095DA0112972A173B07E5
:101E90003CF14A5F5F4F4217530714F1218133270A
:101EA00027FD3095A9014250510984179507C4F0C8
:101EB0002A5F3F4F281739079CF08381811110C09A
:101EC000C69FD001C79FB00D1124A052BC4F948172
:101ED00014968C91981721F0D093D303F092B3020B
:101EE000D093BF0284E58E1510F4D093BF0280E337
:101EF0008D1510F4D093BF02D694D694E694E69450
:101F00000E9DF0011124ED0DF11DE953FD4F80816F
:101F10008C3310F4D093BF020E94E3088091C20278
:101F20008F5F8093C20241CF8091C3028F5F809305
:101F3000C302F0CE41504093C402E3CE8091C5026B
:101F40008F5F8093C502D3CE8091D303811167C088
:101F500081E08093D3031BC02091B402422F50E054
:101F60008091D103992787FD90954817590799F0DB
:101F70008417950724F421502093B40250C02F5F9A
:101F80002093B40230E02817390709F048C084E1F3
:101F90008093B30244C0C091B5028091D203C817A8
:101FA00020F4CF5FC093B5023AC0E091BB0289E054
:101FB000E89FF0011124E052FC4FD2812D2F30E038
:101FC000220F331F21503109DA01A557BD4F8C91E3
:101FD0003AE0632F0E94A031829F202D112490812E
:101FE0009D0F9F5F920F9093D403DA01AE57BD4FC0
:101FF0008C91632F0E94A03191819F5F980F9093E5
:10200000D503C6952C9F202D11242093D6038C9F99
:10201000C02D1124C093D70385E08093C703DF91BF
:10202000CF911F910F91FF90EF90DF9008958F92C5
:102030009F92BF92CF92DF92EF92FF920F931F93E6
:10204000CF93DF931F92CDB7DEB78091C4032BEA05
:10205000829F212D1124269591E1299F9001112421
:102060002D3131055CF090E0039763E070E00E9451
:10207000C23181E1689FE02C112411C00EE027E1FC
:1020800047E063E08EEB94E00E94DA2228EA30E039
:1020900049E064E08EEB94E00E942225E12C10924E
:1020A000C20233E0832E912C41E1D42E5BE1C52E98
:1020B00066E2B62E8091C2029091C603891708F09D
:1020C00045C090E00196B4010E94C2316D9D102D73
:1020D00011241E1958E0510F543690F58C9DF02CA8
:1020E000112463E06F0D0EE027E147E0410F8EEB16
:1020F00094E059830E94DA222091C202B29E90019C
:10210000112428533F4F64E06F0D5981452F8EEB0A
:1021100094E00E9422252091C20230E02F5F3F4FC1
:10212000E091C403F0E02E173F0751F446E0410F61
:102130006F2D6E5F00E129E18EEB94E00E94DA22C0
:102140008091C2028F5F8093C202B4CF60E08EEBB9
:1021500094E00E948C2206E024E540E060E08EEBF3
:1021600094E00E94022361E08EEB94E00E948C22B6
:102170008091C40381111EC08BE18093C7046CE081
:1021800071E08EEB94E00E94792E00E129E146E0B7
:1021900062E08EEB94E00E94DA220F90DF91CF9103
:1021A0001F910F91FF90EF90DF90CF90BF909F9085
:1021B0008F9008958CE18093C70465E171E08EEB08
:1021C00094E00E94792E4AE050E06091C4038EEBC7
:1021D00094E00F90DF91CF911F910F91FF90EF90BE
:1021E000DF90CF90BF909F908F900C94582FFF92CC
:1021F0000F931F93CF93DF9308EC14E0F801108244
:10220000C7ECD4E08CE188836CE071E08EEB94E065
:102210000E94792E8CE0F801808370E1F72EF8821D
:102220006CE171E08EEB94E00E94792E4AE050E080
:102230006091B8028EEB94E00E94582F67E271E043
:102240008EEB94E00E94792E82E1F8018083F8827F
:1022500069E271E08EEB94E00E94792E4AE050E052
:102260006091B9028EEB94E00E94582F67E271E012
:102270008EEB94E00E94792E88E1F8018083F88249
:1022800064E371E08EEB94E00E94792E4AE050E026
:102290006091B6028EEB94E00E94582F67E271E0E5
:1022A0008EEB94E00E94792E8EE1F8018083F88213
:1022B0006FE371E08EEB94E00E94792E4AE050E0EB
:1022C0006091B7028EEB94E00E94582F67E271E0B4
:1022D0008EEB94E00E94792E84E2F8018083F882EC
:1022E0006AE471E08EEB94E00E94792E4AE050E0BF
:1022F0006091B2028EEB94E00E94582F67E271E089
:102300008EEB94E00E94792E8AE2F8018083F882B5
:1023100065E571E08EEB94E00E94792E8091C60213
:10232000482F440F480F440F435F20E930E06BE033
:102330008EEB94E0DF91CF911F910F91FF900C9461
:102340002225EF920F931F93CF93DF931092C20237
:10235000DCE01AE0C6E08091C2028C3008F05EC07A
:102360001092C1025091C1024091C202553108F051
:1023700051C0D59FF0011124E40FF11DE953FD4F29
:102380008081612F0E949431913009F188F0923060
:1023900059F19330C9F5C89F900111242C553B4F3A
:1023A000440F440F652F660F660FE12C01E028C033
:1023B000C89F900111242C553B4F440F440F652FAB
:1023C000660F660F8EEB94E00E9422251DC0C89F09
:1023D000900111242C553B4F440F440F652F660F7D
:1023E000660FE12C02E00CC0C89F900111242C550F
:1023F0003B4F440F440F652F660F660FE12C03E03F
:102400008EEB94E00E9454268091C1028F5F8093EE
:10241000C102A8CF4F5F4093C2029DCFDF91CF9101
:102420001F910F91EF900895CF93DF931092C20206
:10243000C9E0D6E08091C20290E03091B9022091CB
:10244000B802329F90011124821793070CF076C0D6
:10245000C89FF001C99FF00D1124E052FC4F838109
:1024600081110DC02481D29F9001112420573F4F2C
:10247000418160818EEB94E00E94222559C06081E9
:102480006F5F24E041818EEB94E00E949422E09102
:10249000C202CE9FF0011124E052FC4F84818130B2
:1024A000D9F0B8F0823079F1833009F041C0418130
:1024B0004F5F60818EEB94E00E94FD04E091C202C8
:1024C000CE9FF0011124E052FC4F60816E5F41818C
:1024D0002BC041814F5F10C023E0418160818EEBB2
:1024E00094E00E94B722E091C202CE9FF001112435
:1024F000E052FC4F41814E5F23E060818EEB94E01F
:102500000E94B72215C0418160818EEB94E00E9449
:10251000FD04E091C202CE9FF0011124E052FC4F75
:1025200041814F5F60816E5F8EEB94E00E94FD04FD
:102530008091C2028F5F8093C2027CCFDF91CF91E6
:1025400008950F938091B502882309F447C060E095
:102550008EEB94E00E948C2204E02CE040E060E0EE
:102560008EEB94E00E94022361E08EEB94E00E94E7
:102570008C2240E060E08EEB94E00E94FD0443E09A
:1025800060E08EEB94E00E94FD0440E06BE08EEB97
:1025900094E00E94FD0443E06BE08EEB94E00E9427
:1025A000FD0481E08093C2026091C2022091B502D5
:1025B00030E0862F90E02817390784F041E08EEB59
:1025C00094E00E94FD0442E06091C2028EEB94E030
:1025D0000E94FD048091C2028F5FE4CF0F910895A5
:1025E000CF931092C202C9E04091C202842F90E0C2
:1025F0003091B9022091B802329F900111248217C4
:102600009307C4F5C89FF001C99FF00D1124E05253
:10261000FC4F8381811128C08581811125C0809163
:10262000BB02481304C08091BA0281111DC061E051
:102630008EEB94E00E948C22E091C202CE9FF001CA
:102640001124E052FC4F8781823031F0833061F4F5
:102650004181435024E003C04181435022E0608126
:102660008EEB94E00E94B7228091C2028F5F80932C
:10267000C202BACFCF9108958091B502811111C0E5
:102680006AE571E08EEB94E00E94792E6091BC02C5
:1026900070E06F5F7F4F4AE050E08EEB94E00C9467
:1026A000432F08952F923F924F925F926F927F92A5
:1026B0008F929F92AF92BF92CF92DF92EF92FF9252
:1026C0000F931F93CF93DF9360E08EEB94E00E9413
:1026D0008C22E091BB02F9E07F2E7E9EF001112456
:1026E000E052FC4F41814F5F60818281680F6F5FD4
:1026F0008EEB94E00E94FD04E090BB02A090B40237
:10270000B12C7E9C70011124C70180529C4F7C012A
:10271000FC01C281D0E06181772767FD70956F5F12
:102720007F4F882777FD8095982F0E9495301B0159
:102730002C01F501EE57FD4F80811AE0612F0E94B8
:10274000A031682F772767FD7095872F972F0E94FC
:10275000953020E030E040EC5FE30E9421319B01A6
:10276000AC01C201B1010E94FE2F0E946230062F0F
:10277000F7018081BE01680F711D87FD7A956F5F3B
:102780007F4F882777FD8095982F0E9495306B01A9
:102790007C01F501E557FD4F8081612F0E94A0313A
:1027A0009E01220F331F21503109482F4203B001EF
:1027B000439F700D1124882777FD8095982F0E94E4
:1027C000953020E030E040EC5FE30E9421319B0136
:1027D000AC01C701B6010E94FE2F0E946230402F5B
:1027E0008EEB94E00E94FD0461E08EEB94E00E9489
:1027F0008C22C091BB02C090B402D12C7C9EE0011F
:102800001124C052DC4F6981772767FD70956F5F97
:102810007F4F882777FD8095982F0E9495304B0138
:102820005C01F601EE57FD4F8081612F0E94A031BF
:10283000682F772767FD7095872F972F0E94953017
:1028400020E030E040EC5FE30E9421319B01AC01CD
:10285000C501B4010E94FE2F4B015C01EA80F12CFE
:102860008881B701680F711D87FD7A956F5F7F4F73
:10287000882777FD8095982F0E9495301B012C01A9
:10288000F601E557FD4F8081612F0E94A03197012D
:10289000220F331F21503109482F4203B001439FBB
:1028A000700D1124882777FD8095982F0E94953010
:1028B00020E030E040EC5FE30E9421319B01AC015D
:1028C000C201B1010E94FE2F6B017C0120E030E0CB
:1028D00040E85FE3C501B4010E94FD2F0E94623011
:1028E000062F20E030E0A901C701B6010E94FE2FAB
:1028F0000E946230C62F20E030E0A901C501B4017A
:102900000E94FE2F0E946230D62F20E030E040E887
:102910005FE3C701B6010E94FD2F0E9462302C2F99
:102920004D2F8EEB94E00E942B23E090BB02C091D0
:10293000B402D0E07E9C70011124C70180529C4FEC
:102940007C01FC016181772767FD70956F5F7F4F88
:10295000882777FD8095982F0E9495304B015C0168
:10296000FE01EE57FD4F8081612F0E94A031682F3C
:10297000772767FD7095872F972F0E94953020E06D
:1029800030E040EC5FE30E9421319B01AC01C501C6
:10299000B4010E94FE2F4B015C01F7016280712C93
:1029A0008081B301680F711D87FD7A956F5F7F4F3E
:1029B000882777FD8095982F0E9495306B017C01C8
:1029C000C557DD4F8881612F0E94A0319301220FEE
:1029D000331F21503109482F4203B001439F700D2E
:1029E0001124882777FD8095982F0E94953020E04C
:1029F00030E040EC5FE30E9421319B01AC01C70154
:102A0000B6010E94FE2F6B017C0120E030E040E81F
:102A10005FE3C501B4010E94FE2F0E946230062FC1
:102A200020E030E0A901C701B6010E94FE2F0E94FC
:102A30006230C62F20E030E0A901C501B4010E9438
:102A4000FE2F0E946230D62F20E030E040E85FE3A6
:102A5000C701B6010E94FE2F0E9462302C2F4D2F1D
:102A60008EEB94E00E942B23DF91CF911F910F9169
:102A7000FF90EF90DF90CF90BF90AF909F908F909E
:102A80007F906F905F904F903F902F9008950F939D
:102A90001F93CF93DF9305ED13E0C4EDD3E0F8016E
:102AA000408168818EEB94E00E94FD0468816F5F35
:102AB000F80140818EEB94E00E94FD04F801408112
:102AC000415068818EEB94E00E94FD04F801408142
:102AD000415068816F5F8EEB94E0DF91CF911F9141
:102AE0000F910C94FD04CF93DF931092C202C9E0C2
:102AF000D1E08091C20290E03091B9022091B802F9
:102B0000329F90011124821793070CF05DC0C89F7B
:102B1000F001C99FF00D1124E052FC4F80858823FD
:102B200009F44CC0D093C002418146508370481BC9
:102B300060816F5F22E08EEB94E00E949422E0912E
:102B4000C202CE9FF0011124E052FC4F418143505C
:102B500080858370481B60818EEB94E00E94FD04A9
:102B6000E091C202CE9FF0011124E052FC4F41815E
:102B7000425080858370481B60816F5F8EEB94E0CC
:102B80000E94FD04E091C202CE9FF0011124E052A8
:102B9000FC4F4181435080858370481B60816E5F8C
:102BA0008EEB94E00E94FD04E091C202CE9FF00102
:102BB0001124E052FC4F8085815080878091C202B1
:102BC0008F5F8093C20295CFDF91CF9108951092CD
:102BD000C0020E9473158091C002811103C084E07D
:102BE0008093C70308950F93CF93DF931092C2028F
:102BF000C9E0D3E08091C20290E03091B902209107
:102C0000B802329F9001112482179307CCF5C89F18
:102C1000F001C99FF00D1124E052FC4F80856D2F0B
:102C20000E9494319230C9F460E08EEB94E00E94EF
:102C30008C22E091C202CE9FF0011124E052FC4FA1
:102C400004E024E0418160818EEB94E00E94022345
:102C500061E08EEB94E00E948C228091C202C89FBA
:102C6000F0011124E052FC4F9085992329F09150F6
:102C7000908791E09093C0028F5F8093C202BACF99
:102C8000DF91CF910F910895FF920F931F93CF93F0
:102C9000DF9308EC14E0F8011082C7ECD4E08CE17B
:102CA00088836CE571E08EEB94E00E94792E8FE0D2
:102CB000F801808380E1F82EF88262E671E08EEB05
:102CC00094E00E94792E89E1F8018083F8826FE612
:102CD00071E08EEB94E00E94792E8091C602880FFD
:102CE000482F440F440F480F405F20E930E06BE06D
:102CF0008EEB94E0DF91CF911F910F91FF900C9498
:102D000022250F938091B302823009F460C038F419
:102D1000882309F450C0813009F44DC0BBC0853010
:102D200009F47FC0863009F4A7C0833009F0B2C02F
:102D300060E08EEB94E00E948C224091D5034150DC
:102D40006091D403615002E022E08EEB94E00E9497
:102D5000022362E08EEB94E00E948C222091D40347
:102D60004091D50342506FEF620F042F8EEB94E039
:102D70000E942B230091D5036091D4036F5F4FEF26
:102D8000400F262F8EEB94E00E942B230091D50359
:102D90006091D40362504FEF400F262F8EEB94E0EA
:102DA0000E942B232091D4034091D5034F5F6FEFF6
:102DB000620F042F5CC062E08EEB94E00E948C22D4
:102DC0004091D50341506091D40361505EC060E0F2
:102DD0008EEB94E00E948C224091D503415060918B
:102DE000D40361508EEB94E00E94FD0462E08EEB10
:102DF00094E00E948C224091D5036091D4030EEFA1
:102E0000040F2FEF260F415062508EEB94E00E948A
:102E10002B230091D5036091D4032FEF260F4FEFA2
:102E200025C060E08EEB94E00E948C224091D50397
:102E30006091D4038EEB94E00E94FD0462E08EEB7F
:102E400094E00E948C224091D5032091D4030FEF8F
:102E5000040F6FEF620F8EEB94E00E942B23009122
:102E6000D5036091D40321E0260F41E0400F8EEBA3
:102E700094E00E942B230EC062E08EEB94E00E944F
:102E80008C224091D5036091D4038EEB94E00F9196
:102E90000C94FD040F9108950F9360E08EEB94E085
:102EA0000E948C2208E12CE445E064E08EEB94E083
:102EB0000E94022361E08EEB94E00E948C2206E1E6
:102EC0002AE446E065E08EEB94E00E94DA228BE093
:102ED0008093C80481E18093C704E091BB0289E03C
:102EE000E89FF0011124E052FC4F8681811103C05C
:102EF0006FE771E002C067E871E08EEB94E00E943A
:102F0000792E6091BC0270E06F5F7F4F4AE050E025
:102F10008EEB94E00E94432F6EE871E08EEB94E01C
:102F20000E94982E87E08093C7048091BD026AE0DA
:102F30000E949431892F90E0FC013197E930F1052E
:102F400020F4EC5CFF4F0C94173264E971E01AC076
:102F500067EA71E017C06AEB71E014C06DEC71E0D4
:102F600011C060EE71E00EC063EF71E00BC066E06F
:102F700072E008C069E172E005C06CE272E002C074
:102F80006FE372E08EEB94E00F910C94982E0F9308
:102F9000CF93DF9398E0899FE0011124CE5ADD4F53
:102FA00000E020E04E8160E085E994E00E9469291C
:102FB00020E0488161E085E994E00E9469292C8144
:102FC00021954D8162E085E994E00E9469292A817A
:102FD0002A534B8163E085E994E00E94692920E04F
:102FE0004F81698185E994E0DF91CF910F910C9435
:102FF0009A291F93CF93DF938091C703843009F4FC
:10300000CBC130F4813079F0833009F469C1F0C26A
:10301000883009F465C08A3009F4A8C1873009F006
:10302000E7C264E09AC163E08AE794E00E94D82195
:10303000882361F04091C403842F90E00296209190
:10304000C60330E0821793070CF4F7C161E08AE70A
:1030500094E00E94D821882339F02091C403822F64
:1030600090E003970CF0EDC162E08AE794E00E94E3
:10307000D821882359F04091C403242F30E0809157
:10308000C60390E0281739070CF4DFC160E08AE737
:1030900094E00E94D821882321F08091C4038111FB
:1030A000D8C164E08AE794E00E94D821882309F41B
:1030B00006C18091C403811106C088E08093C703D4
:1030C0001092C602FCC025E130E040E050E060E034
:1030D00070E0CB010E94892F6093BD0282E0BEC1E7
:1030E00063E08AE794E00E94D821882351F0809120
:1030F000C602853020F48F5F8093C60202C0109212
:10310000C60261E08AE794E00E94D821882349F052
:103110008091C602882311F0815001C085E0809320
:10312000C60262E08AE794E00E94D821882309F46D
:103130005BC08091C602823051F128F4882349F0A7
:103140008130D1F051C0833061F1843009F443C043
:103150004BC08091B802843010F48F5F01C082E0D0
:103160008093B8028091B7029091B80289133CC055
:1031700081508093B70238C09091B902943020F406
:103180009F5F9093B90230C08093B9022DC08091A7
:10319000B602833010F48F5F01C081E08093B602E5
:1031A00023C05091B7024091B802252F30E0842F00
:1031B00090E001972817390724F45F5F5093B70216
:1031C00002C01092B7028091B70284130DC0415023
:1031D0004093B70209C08091B202833010F48F5F30
:1031E00001C081E08093B20260E08AE794E00E942F
:1031F000D821882309F450C08091C602823029F179
:1032000028F4882341F08130B1F046C0833039F191
:103210008430C9F141C08091B802833010F08150F0
:1032200001C084E08093B8028091B7029091B80207
:10323000891332C024C08091B902823010F08150CD
:1032400001C084E08093B90227C08091B602823029
:1032500010F0815001C083E08093B6021DC09091B0
:10326000B7028091B802992321F091509093B70250
:1032700002C08093B7029091B70298130DC081509D
:103280008093B70209C08091B202823010F0815061
:1032900001C083E08093B20265E08AE794E00E9477
:1032A000D8218111DAC064E08AE794E00E94D82135
:1032B000882329F08091C602853009F4CEC066E0EB
:1032C0008AE794E00E94D821882309F491C16CEE2A
:1032D00074E080E794E00E94FB1F1092880488C18C
:1032E00063E08AE794E00E94D821882351F080911E
:1032F000C602811104C081E08093C60202C0109210
:10330000C60261E08AE794E00E94D821882349F050
:103310008091C602882311F0815001C081E0809322
:10332000C60265E08AE794E00E94D821882319F05C
:1033300084E08093C70364E08AE794E00E94E1217F
:10334000882351F08091C602882319F0813011F052
:1033500003C084E08093C70366E08AE794E00E949C
:10336000D821882309F444C181E064C060E08AE781
:1033700094E00E94D821811174C062E08AE794E051
:103380000E94D82181116DC065E08AE794E00E9417
:10339000D821811166C02CC141E064E08AE794E045
:1033A0000E94F821C091B502882331F0CA3020F480
:1033B000CF5FC093B5021CC1CC2309F45CC0E0917F
:1033C000BB0289E0E89FF0011124E052FC4FD2815A
:1033D0004091B40250E02D2F30E0220F331F2150D6
:1033E0003109DA01A557BD4F8C913AE0632F0E9455
:1033F000A031829F202D112490819D0F9F5F920FFD
:103400009093D403DA01AE57BD4F8C91632F0E9485
:10341000A03191819F5F980F9093D503C6952C9F03
:10342000202D11242093D6038C9FC02D1124C093EE
:10343000D70385E08093C703DBC04D5F4093C4038F
:1034400005CE23502093C4030FCE4F5F4093C40397
:103450001DCE81508093C40324CE81E08093C703A6
:103460002ECFE091BB0289E0E89FF0011124E052E9
:10347000FC4F1086BDC041E061E08AE794E00E9405
:10348000F821811107C061E08AE794E00E94D82109
:10349000882339F08091B402882319F081508093F9
:1034A000B40241E063E08AE794E00E94F8218111D0
:1034B00007C063E08AE794E00E94D821882339F0AE
:1034C0008091B402883018F48F5F8093B40262E078
:1034D0008AE794E00E94D821882359F0E091BB024A
:1034E00089E0E89FF0011124E052FC4F81E08283E3
:1034F0001BC041E062E08AE794E00E94F821882343
:1035000099F0C091BB0289E0C89FE0011124C0522C
:10351000DC4F188169816D5F84E0810F0E94DE04B9
:10352000811102C01F5F188360E08AE794E00E9467
:10353000D821882351F0E091BB0289E0E89FF00197
:103540001124E052FC4F12821AC041E060E08AE789
:1035500094E00E94F821882391F0C091BB0289E099
:10356000C89FE0011124C052DC4F188111506981BD
:103570006D5F812F0E94DE04811101C0188365E018
:103580008AE794E00E94D821882301F18091BA0251
:1035900081111CC08091B502811118C0E091BB025D
:1035A00089E0E89FF0011124E052FC4FC181C35033
:1035B000D0816C2F8D2F0E94DE04811107C06C2FEB
:1035C00083E08D0F0E94DE04882359F066E08AE7CD
:1035D00094E00E94D821882359F01092C60283E01B
:1035E00029CF85E00E94C71786E08093BA02EECF0C
:1035F000DF91CF911F91089580E794E00E94FB1C1A
:10360000882309F405C1109288048091C70390E0D3
:10361000FC013197EB30F10508F0FAC0E35CFF4F95
:103620000C9417320E94F9170C94171081E08093C4
:1036300088040E94F710EAC08091C40381508093EF
:10364000C3030E94310C9091B8029093C50310926D
:10365000B50284E08093B4021092BA021092BC02C8
:103660001092BB028091BE028093E8032091B902C0
:1036700080E0891750F4E82FF0E0EE0FFF1FE852CA
:10368000FC4F208311828F5FF4CF8093C5028AE0C4
:10369000A4C00E944416BAC00E94A1110E94141234
:1036A0000E94F0120E943C130C94E7150E94A11195
:1036B0000E941412E091BB0289E0E89FF0011124FE
:1036C000E052FC4F8681811103C00E94F9170CC0A3
:1036D0000E94620E66E08AE794E00E94D821882367
:1036E00019F083E08093C7030E94EA068091BA0232
:1036F000833070F40E941A07E091BB0289E0E89FD2
:10370000F0011124E052FC4F838181110E94960840
:103710000E94A1120E943C130E94F0128091B502F7
:10372000811176C08091BA02811172C00C9452133B
:1037300080E00E94C7170E94A1110E9414120E94EB
:10374000E3080E9428090C94471581E00E94C717DE
:103750000E94A1110E9414128091B3028F5F809386
:10376000B3020E9481168091B302823019F0873033
:1037700019F008950C94700C1092B3020E94250861
:1037800089E02BC01092C5020E94A1110E94141260
:103790000E941A072091B9028091B802289F9001D7
:1037A00011245091C50240E069E0842F90E0821717
:1037B000930764F4689FF001699FF00D1124E052B3
:1037C000FC4F8581811151E04F5FEFCF5093C502CF
:1037D0004093C40251111CC08BE08093C70308952D
:1037E0001092C0020E9414120E94F3150E94A111AF
:1037F0008091C002811102C00E9496080C947D083D
:103800000E94A1110E9414120E944C170C94F917E7
:1038100008951092C1041092C0048FE992E0909331
:10382000BF048093BE040895CF93CFB7F8948091DE
:10383000F704811127C0EDE3F9E08491E9E2F9E0B2
:103840009491E82FF0E0EE0FFF1FE55AF64FA59197
:10385000B4918C91892321F461E08AE00E94B92D12
:1038600061E08AE00E94802D8CB580618CBD8CB5B2
:1038700080648CBD61E08DE00E94802D61E08BE072
:103880000E94802D8091F7048F5F8093F704CFBF53
:10389000CF9108958F929F92AF92BF92CF92DF9275
:1038A000EF92FF920F931F93CF93DF93EC015C0194
:1038B00086E8A80EB11CD5018C91882309F44DC06F
:1038C0008C3018F41CE0181B01C010E0FE01EA5A0D
:1038D000FF4F81E080836E01BEE4CB0ED11C60E01F
:1038E000C6010E948C224E01E3E58E0E911CD4018C
:1038F0008C9103E0080F9DE2F92E4F2D481B410FDC
:1039000023E0E22E24E560E0C6010E94E92461E0A4
:10391000C6010E948C22F401808103E0080F4F2D24
:10392000481B410F24E560E0C6010E948924FE0186
:10393000E95AFF4F84E080833196D4018C91181BA3
:10394000115D1083CC57DF4F68817981C6010E94D9
:10395000562EF501808181508083DF91CF911F9198
:103960000F91FF90EF90DF90CF90BF90AF909F901E
:103970008F9008950F931F93CF93DF938C01EC01E9
:10398000C25BDF4FCE010E9433226EE476E0CE01AF
:103990000E94562ECE010E9444228CB583608CBDBD
:1039A0008DB58E7F8DBD84E992E0EEEFFFE3099542
:1039B000F801EC5AFF4F108269E276E0CE010E94D6
:1039C000862ECE010E944422065F1F4FC8010E942E
:1039D000A12164E0C8010E94D821811107C062E3DF
:1039E00070E080E090E00E94662CF0CFDF91CF91F4
:1039F0001F910F9108958F929F92AF92BF92EF9275
:103A0000FF920F931F93CF93DF93EC017C0100E8AB
:103A1000E00EF11CF70180809180A280B3800E94AB
:103A2000372C95018401061B170B280B390BB901A4
:103A3000A8015E011FE7A10EB11CF501808190E095
:103A4000A0E0B0E08E0105581F4F84179507A60728
:103A5000B70750F4F80180819181A281B381892B4D
:103A60008A2B8B2B09F06DC0F80180819181A28196
:103A7000B381892B8A2B8B2B09F061C05E01FAE0A0
:103A8000AF0EB11C41E066E0C5010E94F8219E0125
:103A90002B5D3F4F7901882331F065E0C5010E941D
:103AA000D821811185C041E066E0C5010E94F8215E
:103AB000882331F064E0C5010E94D82181118EC0B5
:103AC00041E066E0C5010E94F821882339F048E210
:103AD00064E0C5010E94EA2181118BC0C7010E94E8
:103AE0001E2AC7010E948B2AC7010E945B2BCE01B0
:103AF0000E944A1CCE010E94081E7E013EE4E30E95
:103B0000F11CC7010E944422FE01EC5AFF4F808144
:103B1000811103C0C7010E9433220E94432CF80187
:103B20006083718382839383FE01EB58FF4FC958F2
:103B3000DF4F28813981621B730B7183608380E0C2
:103B40005CC00E94372CF5012081620F711D811D20
:103B5000911DF7016083718382839383FE01EF5887
:103B6000FF4F40815181628173814F5F5F4F6F4F83
:103B70007F4F4083518362837383F80110821182E7
:103B8000128213820E94432CFE01E958FF4F60838A
:103B9000718382839383CE010E94EE20CE010A9628
:103BA0000E94A121CE0148960E94572181E025C0A4
:103BB000C7010E94EA2B61E0680FC7010E94D72B62
:103BC00081EB96E0FE01EC57FF4F9183808388E400
:103BD00032968083C7010E94C12B65CF84EA96E0AC
:103BE000FE01EC57FF4F9183808388E432968083F7
:103BF00067CFCE010E94BA1C71CFDF91CF911F9188
:103C00000F91FF90EF90BF90AF909F908F9008958D
:103C1000DF92EF92FF920F931F93CF93DF93EC010C
:103C20008C8D9D8D892B09F49CC08E01025B1F4FEA
:103C300040E061E0C8010E94902285E5FE01EE5A55
:103C4000FF4F9081891B3596808331961082698D54
:103C5000613009F462C028F0888D653008F074C0C6
:103C60006FC0CE0185960E94212A81E0FE01EA5AAA
:103C7000FF4F80836BE477E0C8010E9441271D8ECF
:103C80001C8EFE01EC5AFF4F108288EAD82E7E016E
:103C90008AE0E80EF11CCE010E94FB1C8823D9F3B8
:103CA00066E976E0C8010E94562E6A8D7B8D4AE057
:103CB00050E0C8010E945F2F61E876E0C8010E94D1
:103CC000562E6D2D62956F7070E04AE050E0C8018D
:103CD0000E94432F66E776E0C8010E94562E64E0FA
:103CE000C7010E94D82181113CC0DA94A1F660E09E
:103CF000CE010E94EA2083B7817F846083BF83B7AF
:103D0000816083BF83B7816083BF889583B78E7FCF
:103D100083BF83B78E7F83BFBECFCF58DF4F48812D
:103D200059816A817B814F705527662777274830F4
:103D300051056105710510F467E009C068E707C027
:103D4000882379F06B5F03C0882359F06FE2C801C4
:103D5000DF91CF911F910F91FF90EF90DF900C9426
:103D60007B2EDF91CF911F910F91FF90EF90DF900D
:103D700008952F923F924F925F926F927F928F920F
:103D80009F92AF92BF92CF92DF92EF92FF920F93EA
:103D90001F93CF93DF93CDB7DEB729970FB6F89473
:103DA000DEBF0FBECDBF998788877C836B831A01E6
:103DB0002C0180E7480E511CF2018081882309F410
:103DC00001C181E0E885F985EA5AFF4F8083E885E3
:103DD000F985EB5AFF4F1082E885F985EC5AFF4FC1
:103DE0001082E885F985108E8F01025B1F4F61E01C
:103DF000C8010E948C22888599858D5A9F4F9A838D
:103E00008983C884D98497E5C90ED11CE884F984D4
:103E1000E8E5EE0EF11C68847984F2E56F0E711C02
:103E2000888599858F589F4F9E838D83A884B984F8
:103E30009AE0A90EB11C88849984E5E28E0E911C4B
:103E4000888599850E94FB1C8823D1F3EB81FC8136
:103E50008491882321F0E981FA81508101C050E0EA
:103E60002DEC36E040E060E0C8015F830E9422252F
:103E70005F812114310439F04CE0450F910160E07D
